:101800003BC06FC054C053C052C051C050C04FC045
:101810004EC04DC04CC04BC04AC049C048C047C074
:1018200046C045C044C0040309041C037700770088
:1018300077002E00660069007300630068006C008A
:101840002E00640065000E03550053004200610045
:101850007300700012011001FF000008C016DC05C3
:101860000201010200010902120001010080320997
:10187000040000000000000011241FBECFE5D4E0EA
:10188000DEBFCDBF10E0A0E6B0E0E0E3FFE102C0C4
:1018900005900D92A636B107D9F710E0A6E6B0E0A4
:1018A00001C01D92AB39B107E1F72FD13FC3A8CFDB
:1018B000A82FB92F80E090E041E050EA60956F5F7B
:1018C00058F42D9138EF82279795879510F084274B
:1018D00095273F5FC8F3F3CF0895EADF8D939D937B
:1018E0000895CF93CFB7CF93DF93C395859BE9F747
:1018F000859B0BC0859B09C0859B07C0859B05C048
:10190000859B03C0859B01C089C06F93C0917E00F9
:10191000DD27CB57DF4F2F9365E5859B03C02F91C4
:101920006F91E6CF0F931F934F9320E040E15F93B9
:1019300000B3047205FB27F93F9350E03BE039C048
:10194000147240642F77012F53501EC0406810B3AB
:1019500014722F7753501FC0406400B32F77047266
:10196000D1F15350000023C0406210B32F7714729E
:1019700091F15350000025C004721027515012F409
:101980005D5F0000115027952C3F10B3C8F614720C
:101990000127015027952C3FC8F64227499300B3F1
:1019A000047210274F73115027952C3FA8F64695C7
:1019B000469510B3147279F00127015027952C3FFA
:1019C00098F66B5A60F3315000B3B0F600C010E4E3
:1019D0001ABF002717C03B503195C31BD04010E4FD
:1019E0001ABF0881033CF9F00B34E9F020917C0028
:1019F0001981110F1213EDCF093651F10D3211F08B
:101A0000013E39F7009383003F915F914F911F9101
:101A10000F912F916F91CAB7C6FD67CFDF91CF911C
:101A2000CFBFCF91189520918300222369F31091A5
:101A30008100112339F534303AF13093810020933D
:101A40007D0010917E003BE0311B30937E001CC076
:101A5000009181000130B4F40AE53091600034FD5A
:101A600014C000936000C1E7D0E013C0052710E068
:101A700000C0000002BB1AC0052710E0221F1DC0D5
:101A800010E021C04AE502C032ED432FC4E1D0E0AE
:101A900032E011B31462959A02B311BB54E220E80C
:101AA00065E320FF052702BB279517951C3FF0F63D
:101AB0006695B8F7B1F720FF052702BB2795179564
:101AC0001C3FD0F62795179517FF052700001C3FF0
:101AD00002BBB0F629913A9519F70B7D109182005F
:101AE000110FC651D04002BB11F010937C0010E4DE
:101AF0001ABF006211B31B7D402F4B7D54E05A95F5
:101B0000F1F702BB11BB42BB7FCF2F923F924F92A6
:101B10005F926F927F928F929F92AF92BF92CF927D
:101B2000DF92EF92FF920F931F93CF93DF9388E1A1
:101B30000FB6F89481BD11BC0FBE909A81E08BBFA7
:101B400082E08BBF8099D1C185B7836085BF8BB799
:101B500080648BBF8D9878946CE0262E312C03E046
:101B600056E4852E58E1952E4AE2642E48E1742E03
:101B700036E2432E38E1532E26E6E22E28E1F22EFD
:101B800094E5C92E98E1D92E86E6A82E80E0B82EDD
:101B900090918100935097FD20C180917E00E101DA
:101BA000C81BD109CB57DF4F80917D008D3209F0E2
:101BB000B8C0983009F00FC123EC209371008AE57A
:101BC0008093600010926A003881832F807629818B
:101BD0008823E1F1B0928000A0927F002330C9F405
:101BE0009B818C812A81203339F48370E82FF0E0C7
:101BF000EE59FF4F808109C0203A11F482D105C00F
:101C0000203C11F46D8185D180E08093690094E0DF
:101C100078C0253011F491E074C0822F8450863052
:101C200008F06EC08A819B8190936C0080936B005A
:101C3000293009F465C09E8190936D008D8182707A
:101C400080936E0037FD61C02FEF60C08A811092D3
:101C50007A00222331F410927B002AE730E092E0F0
:101C60004AC0253019F48093820042C0263081F5A5
:101C70008B81813029F4D0928000C0927F0006C011
:101C8000823031F4F0928000E0927F0092E11CC03B
:101C90008330C9F48A81882331F4509280004092C5
:101CA0007F0094E011C0813031F470928000609226
:101CB0007F009CE109C0823031F4909280008092D4
:101CC0007F009EE001C090E0E0E4E0936A0019C06C
:101CD000283019F424E830E009C0293019F4809341
:101CE000840006C02A3021F42AE730E091E003C0E6
:101CF0002AE730E090E03093800020937F0001C01D
:101D000090E08F81882331F008C0292F80E88093EC
:101D10006A0004C02E81291708F0292F2093610042
:101D20005AC080916A0087FF56C080916D00592F7C
:101D3000891708F4582F851B80936D0060E0882375
:101D400009F461E070916E00E0916B00F0916C001D
:101D500040E036C0CF018F739070892B41F4F89426
:101D600000935700E895789407B600FCFDCF4E5FCE
:101D7000F8948991999121E00C0120935700E895FE
:101D8000112478949F012E5F3F4FC9018F7390708B
:101D9000892B31F0662399F0451788F0772379F085
:101DA000F89485E080935700E895789407B600FC96
:101DB000FDCFF894E1E1E0935700E8957894F901BC
:101DC000451708F4C7CFF0936C00E0936B006623CF
:101DD00011F010926100109281008091600084FFE8
:101DE00078C0809161008F3F09F473C0182F89304B
:101DF00008F018E0811B809361008091710098E8E1
:101E0000892780937100112309F451C080916A00E1
:101E100087FF1EC080916D00811708F4182F811B69
:101E200080936D00A0916B00B0916C00AD01C2E792
:101E3000D0E0212F30E0B9016C0F7D1F05C0FA0101
:101E4000849189934F5F5F4FC617D707C1F727C0AB
:101E500020917F003091800086FF0DC0A2E7B0E0A6
:101E600080E090E0F901E80FF91FE491ED9301960D
:101E70001817C1F708C0D901912FE2E7F0E08D9162
:101E800081939150E1F71150812F90E01F5F0196EF
:101E9000820F931F9093800080937F0008C02A0FC9
:101EA0003B1F30936C0020936B00193060F482E785
:101EB00090E0612F12DD612F6C5F6C3041F08FEF8D
:101EC0008093610004C08FEF809361006EE16093A6
:101ED000600094E180B3847231F49150D9F710928C
:101EE000820010927C00809B53CE12BAF8941BBEE5
:101EF00015BE81E08BBF1BBEE0916F00F0917000BA
:101F00000995E199FECF9FBB8EBBE09A99278DB3CF
:101F10000895262FE199FECF9FBB8EBB2DBB0FB638
:101F2000F894E29AE19A0FBE01960895F894FFCFD3
:061F30005AFF1E9307009A
:0400000300001800E1
:00000001FF
